:0A00000002003EC2A8C28902057A80
:07000B00020571833F7D39FE
:0700130002057DC33F7D39AA
:10001B00C2AB32818882733902142DC477760808FB
:07002B00C2ADC2CAC2CF3210
:10003B0002150A75A8007581C0758911E4F588F55C
:10004B00C9F5C8F5D0F5CDF5CCF5CBF5CA75B8002B
:10005B007580DF7590FF75A0FF75B00F75D8FF75B4
:10006B00C0007820760008B830FA7D007E007F0053
:10007B0020B30ADFFBDEF9DDF7D24580077F0030C6
:10008B00B3EEDFFBD2AF7556FF7558FF7557FF7890
:10009B00B676FFD27AD2001205DF1205C7C2001264
:1000AB0005DF1205C774A61205A174041205A1740D
:1000BB00071205A174801205A1E4D5E0FDE561B43A
:1000CB001107E562B4EE02D245D2957E027F00C2E3
:1000DB0097D297DFFADEF8209002D258C2957E02B3
:1000EB007F00C297D297DFFADEF8209005205802E6
:1000FB00D259205902C2907D08DFFEDEFCDDFAC228
:10010B009474881205A1D2447D02DFFEDEFCDDFA79
:10011B004390F8E4D5E0FDC2937457120D10120D05
:10012B0010120CFD20580E20590B5438B41004D269
:10013B00598002D25A7580DF3058087590EE75B031
:10014B001B80113059087590EF75B00B80067590B8
:10015B00FE75B00F30450302046C9040991206D324
:10016B0075F001743F205807745B20590274061216
:10017B00064874661206481203B278BAE4F608F61B
:10018B00D279C257C25BC25CD256123E30305C0B86
:10019B009042267581C012054A8019123E16D2571D
:1001AB00D25B74401239FF600BB4FF028006B4FEC1
:1001BB00030204D143800FC2D8E4D5E0FD1201F055
:1001CB000460419041C71206D37E031219EE121A36
:1001DB000B7F0A1219A3DFFBDEF11201F00470FA98
:1001EB00D27B022517C2A4D2A47F08E4A2B2205A64
:1001FB0002A2A533305A06C2B6D2B68004C297D239
:10020B0097DFE922021AC21202EF12030F12032C1C
:10021B001203591205DF80FE013E20202020204DC5
:10022B0045504B935088892D31333094202020201A
:10023B002020202020204F4F4F20202288484B4F3A
:10024B0054454B4322202020202020938B2E20200E
:10025B0031362D9F208F41504B4F42419F2C2032E6
:10026B003620202054458B2E202830393529203735
:10027B0034322D30312D313920202020438F414312
:10028B0088814F208741208F4F4B938F4B93202199
:10029B00202017FF01EC00182004000100010108C9
:1002AB00FF04000078203CFF0101340001FF01092D
:1002BB001500008000800000AC83AB8275500012EB
:1002CB000D5B8C838B82E493FFA3600AE493120D86
:1002DB0010DFF9A380F0DEEA020CFD0551E5517049
:1002EB000205522290029D7E0B51C375520175512E
:1002FB00049002A0120DDE51E6E552B583F6E551EE
:10030B00B582F1229002A27E0651C375520275513D
:10031B00A090040051FF75520075510090010080B0
:10032B00D39002BE7E0151C37552007551A090004F
:10033B00E851FF227570FF7571FFE4120E9D755227
:10034B00007551A0020DDE7E0151C3020DDE90023D
:10035B00AF7E0151C37550009002257F78120D5B63
:10036B00E493A3120D10DFF8120CFD7552017551B9
:10037B0000120DDE9002BE75520175510171529043
:10038B0002BE75520175510271529002BE7E01512F
:10039B00C37552007551E89000F151FF9002BE7584
:1003AB00520175510380A0C27C1211107002D27CD5
:1003BB00120FF8121158F56024FC500424FA500364
:1003CB00756009C24A12111F6002D24AC24912114A
:1003DB001A6002D249C2481211156002D248C24FAC
:1003EB0012114C6002D24FC24D12112E6002D24D2F
:1003FB00C24C1211296002D24CC25F12113360023F
:10040B00D25FC25E1211386002D25EC26512110C4D
:10041B006002D265C24E1211476002D24E120FF02B
:10042B00121158900BB878B8A68208A6830208065A
:10043B00E4F5CBF5CA208C0122D5E0F9D5CAF6D567
:10044B00CBF3021A0FE6F70809DFFA221206D312D2
:10045B0019EE12140B304F02D290021A0B30B3016B
:10046B00227581C07F081219A3121A0BDFF8904175
:10047B00F48012904204800D90420E800890420945
:10048B0080039041D37581C0120CFD120D03D20075
:10049B001205DFC2009157D26F1219EE121A0BC25E
:1004AB00AFD29075870280F79041F97581C0120524
:1004BB004A021AC2123E304001229042267581C078
:1004CB0012054A021AC27581C090423E9157121909
:1004DB00EE121A0BD27A12081B301E05123E168032
:1004EB0006301CE2123E23D257D25B74401239FF06
:1004FB00600BB4FE0280CFB4FF0302050B021AC2DD
:10050B009042309157800FC0E09042389157D0E025
:10051B0075F0011206217581C012054C123E1602B0
:10052B001AC290421A80039041EE7581C012054A9F
:10053B00410F9041FF80089041E380039041CE91A1
:10054B0057307F0CC27F74401205A174091205A1AC
:10055B00A27AC0D0D27A12081BD0D0927A201E0574
:10056B001219EE80DC22306E03021A33C2A932C29A
:10057B009032C2AA3243B0C0200003C29222C29171
:10058B0022C0E0C2B792A47403D5E0FDD2B77403C6
:10059B00D5E0FDD0E022F55FB180D3B18CC3B18C37
:1005AB00C3B18CE55F755F0833B18CD55FFAC3B10E
:1005BB008C43900600206C0122021A0F74E3B1A148
:1005CB007418B1A17424B1A17403B1A17401B1A1C8
:1005DB00740880C2B180D3B18CC3B18CD3B18C758C
:1005EB005F86C3B18CD55FFA80C785F08375F064E5
:1005FB0084C0F08583F012062FD0E085F08375F070
:10060B000A84C0F08583F012062FD0E0020629C0C1
:10061B00F0121753D0F0C0E0C412062FD0E0A205A1
:10062B009201C205540FC083C08290069F93D08263
:10063B00D0838009744080058582F0E58330010208
:10064B004480C201C0F0B180D3B18CC3B18CD3B1A3
:10065B008CC0E0E5F0C33325F0D0F03333755F0683
:10066B0033B18CD55FFA755F00741A255F8355F033
:10067B00C36001D3B18C055F740CB55FECB1BCD01A
:10068B00F0E5F0600215F022040280004001080042
:10069B00102000003F065B4F666D7D077F6F777CF8
:1006AB00395E79717408809575F005E572D205D1C4
:1006BB0021E573D205D121E574C12175F004E571F3
:1006CB00D121D13FE570C121E49330E706C0E0B101
:1006DB00DFD0E030E60FC0E075F0057F087408D17D
:1006EB0048DFFAD0E075F00930E50375F00430E42B
:1006FB000375F003540FFFA3E493A3D148DFF92252
:10070B00740975F003D202D20480121218CD740949
:10071B0075F002D202D2048004C202C204ADF0C052
:10072B00E0D26812178FD0E0FF14F5F02490F9C2D5
:10073B0003300416200313E77010EF14600C300223
:10074B00036D60067400D148800FD203300207EFAF
:10075B00146D7002D201E7D12F19DFD522D2D475D7
:10076B00A0FF752300752400208C6D7FFF7EFE7D1E
:10077B00047B00EE52807C40DCFEC2A4D2A44380FA
:10078B000F7C40DCFE7C08EBFA305A08A2B2C2B6F2
:10079B00D2B68006A2A5C297D2974009BFFF04EA42
:1007AB00FF80027F7F0ADCE174082BFBEE23FEDD6A
:1007BB00C2B557028F58EFB5581965576015EF2022
:1007CB00E711E557B47F05FFF5588007EFD218A264
:1007DB00E692198558578F58C2D4220D0E13080470
:1007EB00000C151A0905011611190A0602170F1824
:1007FB000B070314121B1C10FFFFFF305A11C29082
:10080B00D2D4E478B0F608F608F6C2D4D5E0FD22CF
:10081B00C23E208CFB120468305101221207682063
:10082B00184C204403120D03304F39203D362090D5
:10083B0033305A30802ED2D478B630A31476FF08DA
:10084B00762080100816B6000B1876009042208098
:10085B0025B600F078B006B6000A0806B64005903B
:10086B0041C18012C2D41219A375870180A211064F
:10087B0030190C9041CEC2D4120457D23D809190C6
:10088B0007E6E55893F556303D0AB40EE6C23DD265
:10089B003E1205DF24F64002D21AE556B4120712B7
:1008AB00332A7403011BB40C02D21CB40D02D21BED
:1008BB00B40E02D21EB40F13D21D207A0E1219A73A
:1008CB0012140B856483856382E473B41102D22006
:1008DB00B41002D21FB41802D222B41A02D223B41B
:1008EB000A02D227B40B02D226B41902D224B41BAB
:1008FB0002D2250219A712173AAF41BF0001227489
:10090B002F2FF87970E6F71809DFFA22C3FEEC9B5C
:10091B004002C322BC010FE530700B200B08EB64C7
:10092B000D600312093BEEF6080C300B010DD322C0
:10093B00300D031205DFD209C20B78307C007D002D
:10094B00C29CC2ACC2512290001E1206D3D20E75AD
:10095B00F000740D802BD20E740275F0008022D241
:10096B0002D204740475F002120728740475F002A5
:10097B00D20E800DC20E74098007D20E75F0027470
:10098B0009FBAAF0C209C20CC20B111B2051452056
:10099B001A48202745202642301E15203E123009CA
:1009AB000FBB0D02800ABC012C200B29E5307025F2
:1009BB008C418D4030091D3101300B0385407FBBCD
:1009CB000D0F78307970ECFF120450770F09B97F57
:1009DB00FA12177622313BE48022200902313B3098
:1009EB00260DBC0003E43117200E18D20B80142007
:1009FB001A08E431175009E48002E5563117400319
:100A0B00D20C227930EB14FFB40C0C7F09ECC3949D
:100A1B000A6004400229F98FF0EFC39C4011200EAD
:100A2B0006E4120648801BEAC39F40F5E48002E708
:100A3B0009FEC201ED300E01EA6F7002D201EE1217
:100A4B00062F1FBFFFD121957405120ADB30091049
:100A5B00300845C208E570603F24CE403B85701AD4
:100A6B00301B297403120ADB30091030082AC20824
:100A7B00E570600724ED400385701B301B0E74017D
:100A8B00120ADB30090630080F85701CC208301CB7
:100A9B0007120CA55002D208227404120ADB30098B
:100AAB000E30082BC208E57024DC4023857019300A
:100ABB001B167401120ADB30090E300812C208E54E
:100ACB007024A0400A857018C208301C02D208227C
:100ADB00F5F07402C20AD20E8009740675F005D2C5
:100AEB000AC20EFBAAF07C00C209C208111B201A15
:100AFB00218C41200A033008183101300A10E541DE
:100B0B00B4060280092470F8760F08B876FA12172B
:100B1B0076222008032009087C007830D209C2080D
:100B2B00A656080CEC6B7002D20879308AF07F0065
:100B3B00C201300E07ECD39F7002D201EFC39C4071
:100B4B00077408120648800CE709300A04745C80AD
:100B5B00F212062F0FEF6B70D78091C20F75180032
:100B6B00F51985F01A90400612064375F005E51845
:100B7B000412061A12063FE518251A120EB075F06C
:100B8B00021205F5740375F002C20AC20E51EE2073
:100B9B003E54201ED6301B08200822300905802425
:100BAB0030230C0518E518B519C175180080BC3039
:100BBB002434E5187003851918151880AE12189A8D
:100BCB00E57160051219EE80A2E5707006E51870EC
:100BDB00F380051230B450ECE518251A8570F0122D
:100BEB000EA5D20F80BD22C0E01205DF9040ED12A2
:100BFB0006D3D070E57075F00112061A3161C20888
:100C0B00200C0C30090312189AE5706002D20822EE
:100C1B00FA9040F11206D3120C2BB4050092082265
:100C2B00EA75F00012062F111B301E07203E0E7ABC
:100C3B000080ED301A04AA5680E6301B00EA22121F
:100C4B0018CDE57175F003120621E57012062175BA
:100C5B00F0007404D20E318C200C0312189A2291DE
:100C6B004AC208200C08E57045716002D208225177
:100C7B00E5C208301C171217AD90D8071206435166
:100C8B00E5C208301C07121AB07002D208223128B4
:100C9B0031303130313130313031E51B7002C3220C
:100CAB0024ED40FAE51A60F6900C98E51B12175BE1
:100CBB0093FFE51BB40207E51C540370010F0FE50E
:100CCB001AC39F50D92278707F0602045079708026
:100CDB00F774050217D04390E8304413305A077469
:100CEB00801205A18002D2947440D5E0FDC244C2AB
:100CFB0093224390E8C24222D244305A05748802B0
:100D0B0005A1C2942275F008339295C297A296332F
:100D1B00D297D5F0F422E55133E552335407B11095
:100D2B00C3E55133B110E55080DB91E17457B1103D
:100D3B00B11091FDC0E05438B41003D0E02202048E
:100D4B007E91E174543042027456B110B12180B5DA
:100D5B0091E174843042027487B11080B991E174CF
:100D6B00833042027486B1648088B168020D96911B
:100D7B00E174603042027461120D94B135A2E62227
:100D8B0091E174533042027455B17175CB1075CA31
:100D9B0000B13530E70281FDD5CAF6D5CBF302049D
:100DAB007ED2428002B18B7870B14CB110F608DF65
:100DBB00FA81FDD24275500080EDD2427870B15B62
:100DCB00E608B110DFFA81FDD24280F2D2427550B3
:100DDB000080E975CC40A242C0D0B175D0D0924210
:100DEB00C0D0B17A500D15CCE5CCD0D0924270E684
:100DFB0002048DD0D022C242B18B80C0D10112042B
:100E0B006880D0056EE56E7002056F22E56E456F4A
:100E1B006008E56E7002156F156E22D242F5507F99
:100E2B0007787776008080D242F5507F07B1B27891
:100E3B0076E6FF540FF608EF54F0F622D242F55047
:100E4B007877E654F0787646F67F07B1C780E0D224
:100E5B0042F5507F05B1B27874E6FF540FF6087671
:100E6B000008760008EF54F0F622D242F55078775E
:100E7B00E654F0787446F67F05B1C780DAD242F5B6
:100E8B00507F07A1C7D242F55012173A7F02A1B289
:100E9B00D242F5507F02A1C7D242F55085F0707F48
:100EAB0001A1C7D242F5507F01B1B2E57022D24207
:100EBB00F5507F06A1B2D242F5507F06A1C7744D03
:100ECB00800A74488006743E800274C4D242F55086
:100EDB0012173A7F04A1B274C4D242F5507F04A119
:100EEB00C7D242F55012173A7F05A1B2D242F55044
:100EFB007F05A1C7D242F55012173A7F06A1B2D295
:100F0B0042F5507F06A1C7C0E0D19012176DD0E01B
:100F1B00C19BD19085706E85716F22C0E0C0F0D1FE
:100F2B00FF1217ADD0E0D1D7121914D0E080D0C08A
:100F3B00E0C0F0D1EC1217ADD0E0D1D9121914D01A
:100F4B00E080A9C246C247FF1217FFFEEF246FF8DD
:100F5B00E66E600A7870B6FF0608DFFAD24622D238
:100F6B004722EF1217FFF5F0EF246FF8A6F022855A
:100F7B00676E85686F22856E67856F68227550C0B6
:100F8B00A1C57550C0A1AC7F188FF0A4240080615F
:100F9B007F068FF0A42478805874B48052540F20AD
:100FAB002A02240A2324B58004142324DD7F028023
:100FBB004074E9803A74EB803674ED803274EC80C7
:100FCB002E74F8802A74F7802674F9802274FA80C4
:100FDB001E74FB801A74FC801674FD801274EE80F4
:100FEB000E74EF800A74F0800624F1800274EA7F9D
:100FFB0001F5507551007552012274807F40800AB3
:10100B0074F07F02800424007F01F5507551017547
:10101B0052012274067F2A856F83856E8212192CEA
:10102B008FF0A4F550E58224A0F551E583340254EA
:10103B0003F552221475F00C8424E8F55174003436
:10104B0000F5527F14EFA4F5502274AA7F0180178C
:10105B0074A87F018011147F108FF0A424188007CF
:10106B0014232324007F04F550755102755201227D
:10107B00120FE4020DB0113F020DB01161020DB061
:10108B00116B020DB0120F92020DB0120F9B020DDD
:10109B00B012173A120FA8020DB012173A600612CF
:1010AB000FB4120DB022111E020DB01211D9500245
:1010BB00C32211B1D322757110856E72856F738047
:1010CB000A12118D4001C3227571111213D3122D07
:1010DB008874301213F7E4FFFE7D2010510BDFFBF9
:1010EB00DEF9DDF712140BC322122D901047F8E531
:1010FB0071B410F385726E85736F022D9511558047
:10110B004C115B8048120FBC8043120FC0803E1203
:10111B000FC88039120FC48034120FF4802F120FB6
:10112B00CC802A120FD08025120FD48020120FD81A
:10113B00801B120FDC8016120FE08011120FE8805B
:10114B000C120FEC8007120FA480021111120DB0BC
:10115B00E570221105020DB01105020E07E54424BE
:10116B009014FAFF7870E624D05016B40A00501190
:10117B00F608DFF2A84418760F08B880FA12177633
:10118B00D322787079307F07120450E4F56EF56F37
:10119B00F538F539111E7838795174021217D06071
:1011AB0009855138855239120D8B741E2550F55017
:1011BB007F07120DB27870793074071217D0700454
:1011CB0011B1D322120E0E1211D950C8C32278B806
:1011DB00796E74020217D0D2421211EA020D8B758E
:1011EB00520175510322D2D3AD6FAC6E7B017A9055
:1011FB007F00ECC39AFCED9BFD40030F80F4EC2ABF
:10120B00FCED3BFD74042CF55174013DF552EF756B
:10121B00F018A4F550C2D37F182231F1EFFE120D56
:10122B00B0EE120F4E2046033047030204837F18A3
:10123B00120F88E571B56C07E572B56D02D322C349
:10124B0022E56824F04001220204B375F007A424C0
:10125B003E225156020E261475F007A4247D22510E
:10126B0062020E268057F559B408027A07B41002B1
:10127B007A0EB411027A15B412027A1CEA75F0C414
:10128B00120F26E559B40823742A75F0CE120F26D7
:10129B00743175F0D2120F261213751217AD742319
:1012AB00120EFF1219147423120F0AE569456A70A6
:1012BB000C74C8120EB97438120EC1D2380569E518
:1012CB00697002056A22E4F56EF56FF56AF569F54A
:1012DB0018F51912173A7400120F0A7423120F0A19
:1012EB00742A120F0A7431120F0A7407120F0A7440
:1012FB000E120F0A7415120F0A741C120F0A5125C5
:10130B005011E5706008516F856E18856F19120EBC
:10131B000E80EB121340C238E56E456F60118518D5
:10132B006E85196FE56A45696005D238120E0E207D
:10133B003800020F817423120EFF1217AD740E12B8
:10134B000EFF12191474C0120F0C7415120EFF122B
:10135B0017AD741C120EFF1219141217AD74C012B4
:10136B000F011219217400020F0A74D2120ED71238
:10137B0017AD74CE120ED71219141217AD120ED55B
:10138B00021921020DDEC0E0C0E01218CD1217AD1C
:10139B00D0E011A57572017577401217B91217BFFE
:1013AB001217B31215E21217ADD0E011A5757740E5
:1013BB001215761217E402189A7589216005758D3E
:1013CB00FF800B758DFD8006758921758DFA858DD6
:1013DB008BD28E75985022F5993099FDC299E4D530
:1013EB00E0FD227870E671E208DFFA22F5457544DC
:1013FB0070D250C254C255C251C299D29CD2AC22A7
:10140B0075C010C29CC2ACC250C25322C25375F0FD
:10141B0008E4121497D5F0F974031214977412029E
:10142B0014B6309851C0D0C0E0E8C0E0A844D25008
:10143B00E59930561AB4050A7545037544707870F2
:10144B00800DB40604D25C8026B40303754501F607
:10145B000544305313B60D10E545B40104D2558045
:10146B000AB40607D2548003D54504910BD251D050
:10147B00E0F8D0E0D0D0C299C2983292D9C0E074D3
:10148B005B20530274C0D5E0FDD0E022C0F0C2AFA8
:10149B00C3918675F008139186D5F0FAD39186D354
:1014AB009186D2AFD0F022740ED253F545754470AD
:1014BB00C254C255C25175C01075C05022C0E074E1
:1014CB00282053027458D5E0FDD0E022744C2053F1
:1014DB000274B6D5E0FDE4A2DA92E0000000000051
:1014EB00000000A2DA92E10000000000000000A260
:1014FB00DA92E293A2E0220000000100010101C098
:10150B00D0C0E0C0F0C083C08290150291C891E1B9
:10151B00704B91D792F091D792F191D792F291D7DC
:10152B0092F391D792F491D792F591D792F691D7F6
:10153B0092F791D760278882A844A6F005443053D0
:10154B0013B60D10E545B40104D255800AB4060755
:10155B00D2548003D54504910BD251A882D082D0AE
:10156B0083D0F0D0E0D0D053C0DF32D2D312178F5C
:10157B00121793121745787F798FE62778AFF67D90
:10158B000074902DF974802DF8E6FE7F0E78707C38
:10159B0000E68EF0A42C2775F00A84FCA7F008094E
:1015AB00DFEFEC27F77C00940A40020CF709B9AE89
:1015BB00F10DBD0ECC1216C5501A78AFE624F350C0
:1015CB0006FF1216FF80EE1217C578AFE6787FF68E
:1015DB00121776D3C2D322D2D312178F12179312AC
:1015EB001745787079807A007B007F0EE64AFAE720
:1015FB004BFB0809DFF6C3EB6007EA70071217769F
:10160B00D3C2D322787D7D00E61870040DB86FF835
:10161B00ED787F26240DFE79AD747DC39DF8E6F73A
:10162B001819B86FF9770019B98FFA788D7D00E624
:10163B001870040DB87FF8788FEEC3969DFEED60A1
:10164B0018798DE9C39DF8E6F71819B87FF977007B
:10165B0019B97FFA788FE62DF67D0D74932DFB7CEF
:10166B0000EBF87980C268E7B98E0219E4FAE6A2BA
:10167B00689A92685002240AF60908B8AEE9206805
:10168B00030C80DDEBF87980C268E7B98E0219E4B0
:10169B00A26836D4A2E49268C2E4F60809B8AEEAAE
:1016AB00ED2470F8ECF61DBDFFB11217457870797B
:1016BB00901217C978AFEEF6A1C078AFE660167836
:1016CB0090FF7A00E608B400030ADFF8EAFF600532
:1016DB001216FF80E578907D017E00E6086002ED32
:1016EB00FE0DBD1FF6EE940F400904FF1216FF50BE
:1016FB000280E22278AFE6C39F4032F6EFFE248FE2
:10170B00F8E6FB08C3741E9FFF7990120450EEFF9E
:10171B00770008DFFBEBC394054013D378907F1E53
:10172B00740036F6940A4001F6B308DFF3B322C017
:10173B00E01217451217C5D0E022E8789075F0201B
:10174B00760008D5F0FAF82275F00A84C445F02229
:10175B00C0E0C4540F75F00AA4F5F0D0E0540F2587
:10176B00F022787006E60870010622797FF1457841
:10177B00977F08E719C44719F618DFF70978907FA8
:10178B001002045078708002788088F079907F087E
:10179B00E6540FF709E6C4540FF70908DFF2A9F076
:1017AB0080DB7870798080167890798080107870E3
:1017BB007990800A788079708004789079707F10A6
:1017CB000204507402FF1428F8EF1429F9E6C397AA
:1017DB00400670041819DFF522F145F18F789FE66A
:1017EB00760078AFF66003FFD1FF78AFE6789FF60F
:1017FB00F1C5E176D2D3FE1E78707D007C00E60841
:10180B006D2CFC0DDEF8ECC2D322010000000000B1
:10181B00000A00000000000064000000000000E867
:10182B0003000000000010270000000000A086014C
:10183B000000000040420F0000000080969800005E
:10184B00000000E1F50500000000CA9A3B00000013
:10185B0000E40B5402000000E8764817000000106B
:10186B00A5D4E8000000A0724E18090000407A10C1
:10187B00F35A000080C6A47E8D030000C16FF28670
:10188B00237A007E07C3EA9337F7090ADEF822D2E0
:10189B00D3C083C08212178F12174590181578701A
:1018AB00E6FF60067990118CDFFA0874072582F544
:1018BB008250020583B880E81217C5D082D083C24C
:1018CB00D322D2D3C083C08212174590187E789F43
:1018DB000679707A007E07C3EA93FBE79BF7090A48
:1018EB00DEF650EC167970118C18E58224F9F5822E
:1018FB0040021583B88FD91217C512177680BCD248
:10190B00D3787079807F08C322310AE637F608094D
:10191B00DFF9C2D3B322310AE697F60809DFF98063
:10192B00F1D2D3603BFDC37E08330E50FC13FBE4B6
:10193B00FAF9F8C3E5829AF582E5839BF583500AA1
:10194B00E5822AF582E5833BF583B3E833F8E93387
:10195B00F9C3EB13FBEA13FADED9E582898388829C
:10196B00C2D32278707F07E44608DFFC227409801B
:10197B0002740C75F007A42415F582E43418F58372
:10198B00D2D37890E493A3F608B897F8787079904F
:10199B0074071217D0C2D322D26D801CC26B755D37
:1019AB000120580A74601205A1207C0A800020587F
:1019BB000574091205A1C26D206D03205808758CA2
:1019CB0080758A008011206B08758CFD758A80806C
:1019DB0006758CFE758A80755C50D26EC28DD28C6A
:1019EB00D2A922121A0BD26B20581074401205A1E7
:1019FB00755DFF106FB8755D4080B3755D2080AE6F
:101A0B00208CFD2243B0C0C292D312058C7406C346
:101A1B0012058CD5E0F9D312058C7404C312058C16
:101A2B00D5E0F9C26CD29222C0D0C0E0106D642018
:101A3B00583931C1D55D69D26DD26C30926230911B
:101A4B005F7408D5E0FD43B0C0C292D312058C740D
:101A5B0006C312058CD5E0F9D312058C7404C3129E
:101A6B00058CD5E0F9C26CD2928035206B03207CBB
:101A7B0002B290206B08758CFD758A808006758C80
:101A8B00FE758A80D55C19755C50D55D13C290319B
:101A9B00A3800DC26E305802C290C28CC2A9C28DF7
:101AAB00D0E0D0D0327870798074030217D0120650
:101ABB00D3120AE50217AD7581C0D2001205DFC241
:101ACB0000D27A1211E27499120E9085706C8571A6
:101ADB006D307B150225171205DF12173A7572014F
:101AEB007573011206B312081B107EEB90409E51CA
:101AFB00B92022E3201EF2201D3A301C33756601FB
:101B0B00E56612109651B07020304E147420801080
:101B1B00700EBB010B90421412045712081B8097D6
:101B2B00123D6012348C021B750566E566B40AD053
:101B3B0031EE80B59040A151B9201EF8201D0E301A
:101B4B001CEEE412109651B070E60225179040A4DB
:101B5B0051B9201D94301CD8E570B405D3E571B490
:101B6B0005CEE572B405C902229E7581C0C27A7595
:101B7B0063C275641A121151F5651212D1C2661245
:101B8B003E7A7400120EB06002D2707428120EB03E
:101B9B006002D2717450120EB06002D2727478125D
:101BAB000EB06002D2731205DF12173A120719D268
:101BBB00001205DF120719C20075503ED242120DFA
:101BCB005B7F82E4120D10DFFA120CFD85677085C6
:101BDB006871749D120E9B12173A749F120E9B75AF
:101BEB002600752500C20920343C1214B2D20D1206
:101BFB000985C20D12140B300C03021CE6105106A2
:101C0B00301E23021CE912116850151210CC501013
:101C1B0031A7856E70856F71755611D22B021E46DA
:101C2B0012053D021CE930092D752500119A12177A
:101C3B00AD121DC97570FF7571FF74D4120E9B74B4
:101C4B00D18565F0120EA3E565121156F5F074D32C
:101C5B00120EA31217BFE556B4170630377D0221BB
:101C6B0089B41C0D303774300971E525706D022174
:101C7B00F9B4130280EEB4150630375F02212AB493
:101C8B001106752500021E1FB4180F20294D202A9E
:101C9B004A200903302844021E70B41B0F202A3B34
:101CAB00200906202903302832021EF5301F0A2096
:101CBB000904E5256025021F7320230330243230ED
:101CCB00370302213B300913202910202A0D20282D
:101CDB000AA2239230B3923102222C1205472037ED
:101CEB000261B120340912228D121225121DAD6131
:101CFB00ED301B0D200907E5257003021D83021F24
:101D0B009DB4160D2037D43009D1E52570CD0222B4
:101D1B0025301CC7303754E5257050C233300908C5
:101D2B00120ED57493120EE4120ECD1217AD120EC5
:101D3B00C931141217AD120ED131217443120EE4B6
:101D4B003009131217AD7493120ED731215017743B
:101D5B0098120EE4D233743E303305121DB6800355
:101D6B00121DA402205B12054281E92009052028DF
:101D7B000281E6D234021F9D121DA461ED743E90C8
:101D8B004130800C7498904132800574C490412E80
:101D9B00120ED71207160206D3B188D200B188C231
:101DAB000022B196D200B196C20022B18FD200B1FF
:101DBB008FC2002212173A057074CC020E7574C8CC
:101DCB00120EE4120EE2B1BF74D275F000020EA334
:101DDB0085706E85716F74D4120E9B1210B65033D2
:101DEB007F2A120DD97897E6A2E050277418120EAD
:101DFB00D9316EC3601DB1C9741D120EB0F5F074EC
:101E0B00D1120EA3741C120EB0F5F074D3120EA3E4
:101E1B00D228D3229040F51206D312173A0570122E
:101E2B000C6A301E0281E9E556B4140F12095230C8
:101E3B000907E556B41402811681E6B1DB50FA307E
:101E4B002B0FC22B305E0A7426120EB06003021FDA
:101E5B009DE556B4110D1205DF74C8120ED712078B
:101E6B001661F881611205DF906E09120643900628
:101E7B000012064312173A0570305F031214171243
:101E8B00097F300C0281E6205121301E0281E9E5E9
:101E9B004024FC40F074CC120E751217AD74C812AE
:101EAB000ED711CD1215764022A171C251121776A1
:101EBB00E4F573F574F575F57675773074CC120E11
:101ECB007512070B74CC120E5A80B41217E4119AC8
:101EDB00317850D5316E60AD120EE2D22930220826
:101EEB001205DF12071661F881619040FB1206D3D1
:101EFB0012081BC22A202307D22A20240281E612B1
:101F0B0005DF7439202A02747675F0021206487ABE
:101F1B0000120C2B60E7C0E0A22A92E7F5F074D216
:101F2B00120EA3D0E012109C7577401217AD120E53
:101F3B00D511CD1215761217E4119A1217AD120E98
:101F4B00D5302A0431218002311431784002A1713D
:101F5B00316E60FA120EE2D22AE556B41B08120556
:101F6B00DF12071661F88161E565120BF2201E2066
:101F7B0030081B301B18C0E0F5F074D1120EA3D043
:101F8B00E0121156F5F074D3120EA3021F9D81E6D9
:101F9B0081E974D4120E90E5705571B4FF09120EDD
:101FAB00D5E560317E501774C075F000120EA31288
:101FBB000ED51217AD120ED1311431784002A1712A
:101FCB00743E120EE412200E50F474D2120EAE6058
:101FDB000512200E50E8C06EC06F74D4120F1DE5B1
:101FEB006F30E706D06FD06E80111210B6D06FD065
:101FFB006E7970E7600512200E50C3122265D2373E
:10200B00021CEE749F120F12E5717002D322E57160
:10201B00B410002275F005A42452221475F005A407
:10202B00247F22C0E0120ED712196ED0F0600DC0C3
:10203B00F012335BD0E0120ED71233E522C0F01250
:10204B000EFF1217ADD0E0120ED712191402197C25
:10205B0012124C307002110E307102110E307202DE
:10206B00110E307302110E110E110E110E110E11F5
:10207B000E110E110E20301520311220320F110EC1
:10208B00304D0A110E110E110E110E110E110E20E4
:10209B00301020310D20320A749D120F1DC3E567DD
:1020AB00956E12391F749D120F1D203009203106B9
:1020BB002032031212251237F3120E0E203010208D
:1020CB00310D20320AE567B56EE0E568B56FDB12BE
:1020DB0039C51219A3121A0B123DD9120ED1120EB9
:1020EB00E2120ECD74CE120EE4120EC974D2120E81
:1020FB00E4741020300C741120310774122032025A
:10210B007408F5F074C0120EA312173A74C8120EAD
:10211B00C112226574C0120EAE12126F021BC412D2
:10212B00228D121225021FBA78B4A66E08A66F2252
:10213B0078B4866EE608866F462023196003120E6C
:10214B0017121225E570700D74C4904134121D9B4B
:10215B003133021BED120E0EE56EB56707E56FB559
:10216B00680280DA12122550D580DD749F120E9012
:10217B001570E570B4FF021571749F020E9B12224D
:10218B008D121225120ED51217AD120ED112192166
:10219B00743E120EE4120F811221EC317674D212BE
:1021AB000EAE6002317674D4120E90E57120E717F3
:1021BB00C06EC06F74D4120F1D1210B6D06FD06EDC
:1021CB007970E760023176749D120E90E567B570F9
:1021DB0008E568B57103021BB1120E173133021CEF
:1021EB00EE12173A7448120EE4744D020EE47F4857
:1021FB00E556B413027F4DEF120EE4120ECD1217FB
:10220B00AD120EC91219141217AD120ED1121921DB
:10221B00400531EC021D71021D83D23290412C809E
:10222B002090412820300390412A1206D312081B1C
:10223B00301E03021BB1201C06752600021CE60192
:10224B005BE565120BF2301CF0F5F074D1120EA3A6
:10225B0074C490412C121D9B80E512124C7F1812F6
:10226B000F8D856673856C71856D72120F7A1211E5
:10227B00F1120F6D120E0112138E3133120E0E026C
:10228B000F81120F7A020E171217AD7400120EFF88
:10229B000219217581C0C27AC20DC266C264904018
:1022AB00B51206D37563C275641A12081B75639E4B
:1022BB00756422E556B401080223361219EE80D359
:1022CB00B40303022437B404F20224529040C9121F
:1022DB001AB9E4120E8AE5705571557104201C0170
:1022EB00E422E5599041177E07600590411C7E045E
:1022FB008E5A1206D3300F0C8E507F03120DAC7416
:10230B0006120724740675F005C20A120AEE201E87
:10231B00D1201B051219EE80C92008072009F520D2
:10232B0046F222855A507F03020DC551D760291200
:10233B00173A7400120EE47404120F0A123EEE9058
:10234B0040B91206D37818120CD8740A120EC112A7
:10235B0006B312081B201B0241C69040BF1206D3C6
:10236B00300F0A7400120ED7740812072474087504
:10237B00F007C20A120AEE201EE0201B051219EE0E
:10238B0080D82008082009F5300FF2800574001260
:10239B000EE475590051ED055951ED9040C91206E7
:1023AB00D3120C7A200808301B001219EE80ECE5D2
:1023BB0070557155720460F27550107F06120DC581
:1023CB0012409312400E419E1205DF9040E1E559F9
:1023DB0060039040E41206D312173A7572017573BD
:1023EB00017918120CD11206B3120A5330080FE5FB
:1023FB005923232448F8A61A08A61B08A61C221248
:10240B0005DF9040E7E55960039040EA1206D312CE
:10241B00173A120C4AC208E5704571600EE5592354
:10242B00232448F8A67008A671D20822D2617559E8
:10243B000071D320080820640241C602261C0559EE
:10244B0071D33008F18011C261755900910A3008BF
:10245B00E50559910A3008DE7848794C7403206100
:10246B0001141217D0600250CD9041261206D312E0
:10247B00081BD260E5566005C2601470B912344374
:10248B0020640E51D7700241C6124093123AEC41B0
:10249B009E124093206105123C7D8003123C370253
:1024AB002517124093023BB11205DF75F009743901
:1024BB0012064812173A120C4A301B0C85704885CD
:1024CB007149E5704571700302261C124093023B63
:1024DB00F81205DF75F009745E12064812173A748C
:1024EB0008120724740875F007C20A120AEE201EA0
:1024FB00E0201B0302261C3008FA857048857149C1
:10250B0085724A85734B124093023CF17581C0C2B0
:10251B007AC20DC2661203B29040A71206D375633E
:10252B00C275641A12081B756317756425301B037B
:10253B00022621E556B413030230D3301A030227C7
:10254B00BF302207D260122A8B80C1301F030228B2
:10255B0037C22A202305302405D22A022A3A3020FA
:10256B00030228953025030227E8B41503022856E9
:10257B00B41603022AD0B40B0302261CB4170302B1
:10258B002BF9B41403022DDCB41C06022D430226D6
:10259B001CB40CFA905B0412064312081BE556B4EC
:1025AB001103022C12B4130302261CB41C030226C3
:1025BB001CB40B0302261CB41B03022C6CB41A03B1
:1025CB00022C5AB4180302261CB40003022C7EB44E
:1025DB000103022CA2B40203022CD8B4030302267B
:1025EB001CB40403022B64B4050302261CB41003B1
:1025FB0002261CB4060302261CB41403022CB4B42A
:10260B00150302310CB40903023144B4080302313F
:10261B004A1219EEA117207BF89040AC1206D31288
:10262B0012D112081B201B3B301C03022710E5564E
:10263B00301A056003023174301F030231803025DC
:10264B000280CE30220302318EB4150280C3B41146
:10265B000280BEB40B0280B9B40A0280B47002804F
:10266B00B080AE9040AF1206D312081B301B02A1F4
:10267B0017301C23D257756600123E3012348C1261
:10268B004093123A841211E27499120F121211EA4A
:10269B00D242120D75A117E556B40906D26091B35B
:1026AB00A117B40606C26091B3A117B4050491DC5F
:1026BB00A117B40404D2648152B40304D2648137E9
:1026CB00B402091226F4501F91ADA117B4000D12DC
:1026DB0026F45013124093123D30A117B40B08127D
:1026EB004093123BE1A117C11C9042511206D31229
:1026FB000AE5E570B4120CE571B43407E572B45613
:10270B0002D322C322D257756600123E3012348C8C
:10271B00124093123A7DA1179041B51206D31217AE
:10272B003A0570120C4A201B051219EE80EAE5716E
:10273B00B56A00400970F2E569B5700040EBE4F54D
:10274B006EF56F857018857119F51B751A01E51BF0
:10275B00B5194DE51AB51848121225E570F55990C3
:10276B00412E6012B41003904128B4110390412AFA
:10277B00B4120390412CB40802A117C083C082127B
:10278B000ED5120716D082D0831206D312081B2047
:10279B001B051219EE80C1E55970DE120E0E80B8C2
:1027AB00121225120E0EE57060F6051AE51A70026C
:1027BB00051B809AF5599041091206D3E55960061D
:1027CB0075F00812062F120C7A2008071219EEE585
:1027DB005980E1E559120F9B120E07A117740112D4
:1027EB000BF2201EF8201B051219EE80F03008F8B2
:1027FB00F5591205DFE55975F00912061AE559125C
:10280B001156120C1B201B08201C1E1219EE80E205
:10281B003008F8F570E559121011120E070559E53D
:10282B0059B464CE75590180C90225171211511282
:10283B000BF2201EF7201B051219EE80EF3008F863
:10284B00F570120FA4120E070225171205DF904028
:10285B00B21206D31204BF123E7A755900755A0094
:10286B0075F007E5590412062F855AF07428120BE0
:10287B0066201C0302261C123EA4E55A2428F55A96
:10288B000559E559B404D90225179040F51206D322
:10289B0012173A0570120C6A3020329040FE120665
:1028AB00D31214B212081B12140B1051082020DA89
:1028BB001219EE80D512116850F612118D50F112CB
:1028CB00173A856E70856F711219A780C83008E0B2
:1028DB00301BDD85706E85716F1211D940D21210CD
:1028EB00B17F2A120F889040F91206D374D8120EBA
:1028FB00D7120716120985201B051219EE80E73037
:10290B00090812189A74D8120EE474DD120EAE1266
:10291B000BF2201EF52008051219EE80ED301BF886
:10292B00F5F074DD120EA31205DF74DC120EAE127D
:10293B000C1B2008051219EE80ED301BDBF5F07433
:10294B00DC120EA39041591206D374E6120EAE544C
:10295B000175F00012062F12081B201B18201A05F8
:10296B001219EE80DFE556B4020050F4F5F074E670
:10297B00120EA380CF9041721206D374E7120EAEE3
:10298B00F559540175F00012062F12081B201B1E5F
:10299B00201A051219EE80DDE556B4020050F4E55D
:1029AB0059C2E04556F5F074E7120EA380C790406C
:1029BB00F51206D37550C07F18120DAC7F18120D8F
:1029CB00D9741875F000120B66201C051219EE80D5
:1029DB00DD7F18120DC07550C07F18120DC59041C8
:1029EB00AA1206D31214B212081B12140B10510E9A
:1029FB00202415903F00201B1F1219EE80E01211AE
:102A0B006850F6903100800B787076FF08B877FA33
:102A1B0090390074DE120E8812064312081B301C0C
:102A2B00D87F2A120F8D12101E120E0702251712B5
:102A3B0005DF903909202A037583761206437A0144
:102A4B00120C2B201B051219EE80E460F9F5597559
:102A5B00F00812062FE55912109C12096A301BE67A
:102A6B00200CE3300908E559120FA8120E070225B6
:102A7B00171205DF90DF091206431206B3020A5341
:102A8B00123EEE851A72851B73851C74517C2008CF
:102A9B00051219EE80EA1205DF90780912064385BC
:102AAB0019718518701206C6120AA43008E3123F7A
:102ABB0025123F250225179040D01206D375F0073B
:102ACB00E56E02062F756E0151C212173A12096A92
:102ADB00201B08201C051219EE80ED200CF8E412C7
:102AEB000EE6123EEE7F40120F88E56E123F8D050B
:102AFB006EE56E6405600280CF12173AE4120EE6A3
:102B0B00123EEE7F40120F88E4123F8D02251774A0
:102B1B0001120BF22008051219EE80F3301BF88519
:102B2B007059E5591210817F14120DD975F0097483
:102B3B0039120648E55912061A741475F000120B77
:102B4B0066201C051219EE80D97F14120DC0E559B1
:102B5B0012103F120E0702251790416A1206D37509
:102B6B005901E55975F00012062F12081B301A0D8A
:102B7B00E55670051219EE80E0F55980E5301BF42F
:102B8B00E5591210867F10120DD9741090416A12FC
:102B9B0006D3E55975F00712062F741075F0001265
:102BAB000B66201C051219EE80D67F10120DC0E5A6
:102BBB0059121061120E07022517122BD6C3201EB5
:102BCB0004301B02D3221219EE80EFE57060027401
:102BDB000175F00012062F12081B201A062212197B
:102BEB00EE80E8E5566003B401F4F57080DD9041AA
:102BFB00361206D312111071C550F3120FBC120E00
:102C0B00071203B20225179041391206D312111580
:102C1B0071C550F3120FC080E590413D1206D312DF
:102C2B00111A71C550F3120FC880D390414112068F
:102C3B00D312111F71C550F3120FC480C1904145BF
:102C4B001206D312114771C550F3120FE880AF90E3
:102C5B00414E1206D312112971C550F3120FCC80BD
:102C6B009D9041491206D312112E71C550F3120FCC
:102C7B00D0808B9041531206D312113371C550F390
:102C8B00120FD481099041801206D312110C71C519
:102C9B0050E112105B81099041591206D312113881
:102CAB0071C550F3120FD881099041A01206D312AF
:102CBB00110871C550F31210558109904177120616
:102CCB00D312107B71C550F3120FE4810990415F51
:102CDB001206D3E4F559E55975F00012062F1208C8
:102CEB001B301A0CE556B40800500B85565980E67C
:102CFB00201EDA201B051219EE80D2E559123D87F2
:102D0B000225179041641206D3121142F559E55969
:102D1B0075F00012062F12081B301A0585565980C4
:102D2B00ED201EDF201B051219EE80D7855970127E
:102D3B000FE0120E070225179041B91206D3E5607A
:102D4B0075F00012062F12081B301A10E556B4044A
:102D5B000050051219EE80E0F56080E2301BF41292
:102D6B000FF8856070120E0702251790410C1206A2
:102D7B00D312114C71C550F3120FEC81097F301235
:102D8B000F6D0213EE7430020F4E787479707F2A38
:102D9B001204507870E67005B8700780071230B4D3
:102DAB004002C32208B888ED789A76000876CA08E4
:102DBB00769A08763B7888799A74041217D050E289
:102DCB00788CB6050050DB08E660D7249C40D3D343
:102DDB0022C2569000201206D31213D3E4D5E0FD85
:102DEB007570F87571F9B1887840D9FED8FC12115D
:102DFB00081213C4751CFF751DFF751E007430126D
:102E0B0013F73051FDC251B1902047132046108566
:102E1B007050857151E572B4FF08742002251702BA
:102E2B002EC0F55220E744751E00755A127F2CE513
:102E3B0052601BB4020CE551B4980050117552004E
:102E4B00800C500AE551B404004003755200120D7A
:102E5B00B0B188E550242CF550500B75500005513E
:102E6B00E55170020552D55AC48092E573F559B1FC
:102E7B0095E55220E618503D85506E85516F121125
:102E8B00D9403212101E120E07751E00800E20E55F
:102E9B000302304830E41E30E31B800D7570F07573
:102EAB00710F7F021213EEC108E559B4201EE570B5
:102EBB00123095400B7570557571AA751E0080E226
:102ECB00E55012308750EE12101180BAB4211578EC
:102EDB00707F181230BF50DDE550B4050050D6128C
:102EEB000F9280A2B4220CE550B40A0050C7120F07
:102EFB009B8093B4230CE57012308750B8120FA44B
:102F0B008084B42413D22A12309950A9E550B40A04
:102F1B000050A2120FA8C191B42504C22A80E8B4B4
:102F2B002613123099508EE550608AB405005085F7
:102F3B00120FB4C191B42707120FBCC191C1C0B419
:102F4B002811E570B4040040F4B40A0050EF120FDE
:102F5B00F8C191B42905120FC0C191B42A05120F03
:102F6B00C8C191B42B05120FC4C191B42C05120F1B
:102F7B00E8C191B42D05120FECC191B42E1FE57071
:102F8B005407B4050050B6E570C45407B40500509F
:102F9B00ACE550B4040050A5120FF4C191B42F0549
:102FAB00120FD0C191B43005120FCCC191B43105C1
:102FBB00120FD4C191B43207120FD8C191C1C0B452
:102FCB00330CE570B40A0050F4120FDCC191B43429
:102FDB000CE570B40A0050E5120FE0C191B4350551
:102FEB00120FE4C191B4380512105BC191B43618BD
:102FFB0078717F031230BF50C4E55060C0B4050038
:10300B0050BB12106B022E91B4371678707F1012D2
:10301B0030BF50A9E55012308E50A2121061022E13
:10302B0091B4391678707F141230BF5090E550125E
:10303B003087508912103F022E91022EC0500B8503
:10304B00506E85516F1211D95003022EC012101EF3
:10305B00E551B51C09E552B51D04E51E700C120DAA
:10306B008B85511C85521D751E017F2A120DC7E5DC
:10307B00597006120DDE751E00022EA7C36003B435
:10308B00640022C36003B40A0022B4050022E57079
:10309B00B4A0005013540FB40A00500CE571B4A047
:1030AB00005005540FB40A0022B420005002B32282
:1030BB00B4F0002288F0E611B440067008E8B5F0D1
:1030CB000508DFF2D322C3229041BD1206D37559F6
:1030DB0000E55975F00012062F12081B201B11E595
:1030EB005660081460051219EE80DD85565980E193
:1030FB00E559123DB00225177872798274030217D5
:10310B00D075F000D5E0FDD5F0FA7B00C2B17F0899
:10311B00D5E0FDDFFB20B01AD2B17F08D5E0FDDF93
:10312B00FB30B00EDBE69041931206D312081B0264
:10313B002517D2B190419A80F01202EF0225171297
:10314B000359022517E4F56EF56F751EFF751FFF0A
:10315B00F550FFD242120D5BE4120D10DFFA7F081F
:10316B00E4120D10DFFA020CFD7559001240931298
:10317B003A76022517C260755901124093123A6BC9
:10318B000225171205DF7401120BF2200803022629
:10319B001C301BFAD260121753F559124093123A96
:1031AB006B022517787479707F04120450E4F57460
:1031BB00F575F576F577221217AD12173A7887E683
:1031CB007600B430081217BF7577008017B420054E
:1031DB0075701080096004057180037571101215EC
:1031EB00761217E402189A90418C1206D312081B20
:1031FB00201C0302261C9041A81206D330381775E9
:10320B0051A0755200120D8BE4120E92E56CB57045
:10321B0008E56DB57103022517E4F518F519751A54
:10322B002AF51B751CB8751D0B755AA0E4F56EF5C8
:10323B006F751EFF751FFF755200855A51D24212D2
:10324B000D8BE55AB4A00A856C70856D71E4120E76
:10325B009B1211F1120DB0E57070697885E620E7CD
:10326B00631879181217CE405B7884791A1217CE2F
:10327B00401D781C79841217CE40107884791E1269
:10328B0017CE50407884861E08861F803780C27800
:10329B0084E6C3951875F006A4F559787C79707F90
:1032AB0005120450E4F575F576E57454F0F5775393
:1032BB00740F31C21217ADE559120EFF121914E536
:1032CB0059120F0A120E0EE56EB567C1E56FB568A0
:1032DB00BC755200855A51D242120DDE055AE51AC1
:1032EB00F518851B19242AF51AE4351BF51B781CD8
:1032FB0079181217CE400B781E791A1217CE50DCA4
:10330B00413741219041851206D312081B201C0323
:10331B0002261C9041A81206D312032C0225177506
:10332B005400021A0B121753C0E0C412333BD0E007
:10333B00540F2430F5F0E554B41801222430F8A6CC
:10334B00F0055422742080ECFF7420713FDFFA22C9
:10335B00E493A3700122B420005004715380F1B4A4
:10336B00F00040027420713F80E67970E7B42000D2
:10337B00500474208005B4F00050F709713FDFEC66
:10338B0022E5717133743A713FE570809BE5727180
:10339B0033742E713FE5737133742E713FE5748076
:1033AB0087718C714F80E6C210C212803D12176D6F
:1033BB007872760008B878FA1218CD7404C210C26D
:1033CB00128027E5777002714FE577C4F5F0740929
:1033DB00D210D2128014740E80027409C0E012183D
:1033EB00CDD0E075F002D210D212C0E0C0F01217AF
:1033FB008FD0F0D0E0ADF0FF246FF9C21130121472
:10340B00201111E7700EEF14600A3010036D600489
:10341B00714F8010301008EF6D7004742E713FD215
:10342B0011E7713B19DFD622E5717133742E713FB1
:10343B00E57071337425613FD25674010213C4EFEA
:10344B00FC7570027871ECFFFE7D00E62DFD08DE49
:10345B00FAEDC4540F2430F608ED540F2430F6085F
:10346B0076030F0F0F0F1213EE22EB1213F712133B
:10347B00EE7630087630087630087630087600081D
:10348B00229143755B007570027871743112351B94
:10349B00123506E56612352F12351A123538E566E8
:1034AB006007121086E570702578707F2812351A28
:1034BB00DFFB12351A1234F912353874131239FF37
:1034CB007873123A5F123A5FA2E19277E422787036
:1034DB007970E70912351BB980F87F1880CF540F2C
:1034EB00B40A004004243780022430F60822E55B3E
:1034FB00C491E9E55B91E976030822743012351B20
:10350B00743012351B743012351B743012351BE4BA
:10351B00F608255BF55B22540FB40A004002240722
:10352B00243080ECC0E0C4B122D0E080EAE8C39440
:10353B0070FF0213EE7F28B11ADFFC2212173A85B7
:10354B0061708562710561E561700205621218CDCB
:10355B001217AD78707981E719B122E7B12F80AFDF
:10356B0075F000B46400400605F0946480F5C0E08B
:10357B00E5F0B122D0E0121753B12F80927870741E
:10358B0000B12FB11A7400B12F7420B12FB11A747E
:10359B0029B12FB11AB138B1477F05B142B140B152
:1035AB001A808A7870B12FB11A7400B12F7420B1C0
:1035BB002FB11AE4B12FB11A80DB78707405B12FDB
:1035CB00B11A7400B12F7420B12FB11AE4B12FB11D
:1035DB001A80C278707406B12FB11A7400B12F74AF
:1035EB0022B12FB11AE4B12FB11A80A978707407E8
:1035FB00B12FB11A7400B12F7420B12FB11A7432DC
:10360B00B12FB11A808F78707408B12FB11A740072
:10361B00B12F7420B12FB11A7432B12FB11AA1A0EE
:10362B0078707410B12FB11A7400B12F7420B12FB0
:10363B00B11AE4B12FB11AA1A078707412B12FB1E5
:10364B001A3077127435B11B7430B11B7430B11B47
:10365B007430B11B80107430B11B7430B11B7432D9
:10366B00B11B7430B11BB11AE4B12FB11AA1A07800
:10367B00707413B12FB11A7430B11B7430B11B7449
:10368B0032B11B7430B11BB11AE4B12FB11AB1387E
:10369B00B1477F05B142B1383033077493120ED75F
:1036AB008003120ED1712A71E5740A1239A77F1E9D
:1036BB00B11ADFFCB11AA13878707414B12FB11A9A
:1036CB007430B11B7430B11B7432B11B7430B11B2D
:1036DB00B11AE4B12FB11AA1A024157870B12FB192
:1036EB001A7430B11B7430B11B7432B11B7430B10E
:1036FB001BB11AE4B12FB11AA1A0C0E07870749974
:10370B00B12FB11A7430B11B7430B11B7432B11BB1
:10371B007432B11BB11AE4B12FB11AB138B1477F72
:10372B0005B142B138D0E0C0E0FF123748D0F07499
:10373B0028C395F06003FFB142B11AA138787079B4
:10374B0030E709B11BDFFA22C0E078707411B12F9A
:10375B00B11AB138E420301120310E20320B74D362
:10376B00120EAEB405004001E47870B12FD0E0B179
:10377B002FB11AE4B12FB11AB138B147A138787013
:10378B00121753B12FB11AA138120ED7712A71E546
:10379B00787079307F00E709B420030F8002B11BEA
:1037AB00B93AF3EF60051FB11A80F8B11AB11AA13B
:1037BB0038203028203125203222120E5A712A71DE
:1037CB00CE787079307F00E709B420030F8002B107
:1037DB001BB93AF3EF600B1FB11A80F878707F0AB0
:1037EB00B142B11AB11AA138C2282030352031327A
:1037FB0020322F74D4120E90E571046025D228C0AC
:10380B006EC06F85706E85716F1210B6D06FD06EF3
:10381B0012332A7F187970E7600812337774181205
:10382B003705742212375374D1120EAE123789201A
:10383B00301220310F20320C74D4120E90E571042B
:10384B00D228700512173AC2281218CD1217AD786C
:10385B00707981E71912352FE712352F7F03123557
:10386B004212353878707F0612354212353874CCD7
:10387B001237BC74C420300820310520320274C8C2
:10388B0012379478707F0612354212353820307912
:10389B0020317620327374D2120EAE606C74D21259
:1038AB000EAEA2E7922A7420302A0274A01237536C
:1038BB0074D1120EAE1237897870E41235227F065E
:1038CB0012354212353874D2120EAE12109C1233CE
:1038DB002A1234337870E53012351BE53112351B63
:1038EB00E53212351BE53312351BE53412351B124D
:1038FB00351A12353874CC1237BC74C81237947819
:10390B00707F06123542123538221561E561B4FF1E
:10391B0002156222123443755B0075700278717464
:10392B005312351B1235063030047432801030318F
:10393B0004743380093032047431800274301235D0
:10394B001B12351A740412352F12351A1235381210
:10395B00173A749F120E9012355812353875610054
:10396B0075620030700574011235AE30710574024A
:10397B001235AE30720574031235AE307305740414
:10398B001235AE12362B31151235881235C531155D
:10399B001235F71235DE3115123611227870793067
:1039AB00FE7F00E709B420030F800312351BDEF303
:1039BB00EF60061F12351A80F722787012364420FA
:1039CB003028203125203222304D1974001236E474
:1039DB0074011236E474021236E474031236E47482
:1039EB00041236E412367A1236C378701234F91296
:1039FB003538740C1213F77F007E007D10C2501007
:103A0B00511ADFFBDEF9DDF72050EC12140B305BA3
:103A1B000474FF8027C25BC25702050BE570B40527
:103A2B000E30570474FE8014C25BC2570204D1B42B
:103A3B0002D9787A123A5F6003305705C257C25BDE
:103A4B0022C257C25B020512E60824D0B40A00401A
:103A5B00029427225153C4C0E05153D0F045F022B9
:103A6B0075F0047403A26092F3801375F004740272
:103A7B00800C75F0047401800575F0047400C0F0BF
:103A8B00C0E01204BF755B007570027871745F1231
:103A9B00351B123506D0E012352212351AD0E01242
:103AAB00352F12351AE55912352F12351A1234F9F2
:103ABB00123538740C21FFE4120ED912178F12171E
:103ACB00AD798478707F00E719B40F030F80031270
:103ADB003522B97FF2EF60061F12351A80F70235D7
:103AEB001A1204BF755B007570027871744212353F
:103AFB001B12350612353851C27400206102740254
:103B0B003060010412352212351A12353820612A21
:103B1B0012173A8548708549711218CD1217AD7876
:103B2B00707981E71912352FE712352F12351A12DA
:103B3B00351A12351A12351A80167870E548123577
:103B4B002FE54912352F742012352FE54A12352FE8
:103B5B0012351A12353820612A12173A854C7085A6
:103B6B004D711218CD1217AD78707981E719123596
:103B7B002FE712352F12351A12351A12351A123544
:103B8B001A80167870E54C12352FE54D12352F74CF
:103B9B002012352FE54E12352F12351A1234F91229
:103BAB003538740C21FF1204BF755B0075700278F9
:103BBB0071745812351B1235061234F912353874DC
:103BCB001321FF1204BF755B007570027871745975
:103BDB0012351B02350671CEE41235227F131235D6
:103BEB001ADFFB1234F9123538741321FF71CE74BE
:103BFB0001206002740712352212351A1235381261
:103C0B00173A8548708549711218CD1217AD787027
:103C1B007981E71912352FE712352F7F0D12351ADF
:103C2B00DFFB1234F9123538741321FF71CE740493
:103C3B003060010412352212351AE54812352FE592
:103C4B004912352F742012352FE54A12352F1235B4
:103C5B001AE54C12352FE54D12352F742012352FE6
:103C6B00E54E12352F12351A1234F91235387413FA
:103C7B0021FF71CE74023060010412352212351A05
:103C8B0012353812173A8548708549711218CD12C2
:103C9B0017AD78707981E71912352FE712352F128E
:103CAB00351A12351A12351A12351A12351A1235EF
:103CBB003812173A854C70854D711218CD1217AD0D
:103CCB0078707981E71912352FE712352F12351AD3
:103CDB0012351A12351A12351A12351A1234F91204
:103CEB003538741321FF71CE740612352212351A32
:103CFB0012353812173A854870854971854A728595
:103D0B004B7312178F1217AD78707987E71912352D
:103D1B0022B97FF87F0A12351ADFFB1234F91235FC
:103D2B0038741321FF1204BF755B00757002787134
:103D3B00745A12351B1235061234F91235387413B6
:103D4B0021FF1204BF755B007570027871745712F6
:103D5B00351B023506B14D740012352212351A127D
:103D6B00351A12351A740012352F740812352F12AA
:103D7B00351A1234F9123538741321FFC0E0B14DE6
:103D8B00D0E012352212351A12351A12351A740078
:103D9B0012352F740312352F12351A1234F91235CE
:103DAB0038741321FFC0E0B14DD0E012352212352B
:103DBB001A12351A12351A740012352F7406123571
:103DCB002F12351A1234F9123538741321FF1234AD
:103DDB0043755B007570027871743812351B1235A0
:103DEB0006740012352212351A745012352F123503
:103DFB001A741912352F12351A740112352F123508
:103E0B001A1234F9123538741321FF1234437870B7
:103E1B00740112351B023538123443787074041256
:103E2B00351B023538C25C12344374011213F77F11
:103E3B00007E007D05205C06DFFBDEF9DDF712144A
:103E4B000BA25C22C0E0C0F0755B0075700278714C
:103E5B00745C12351B123506D0E0123522D0E012FD
:103E6B00352F12351A1234F9123538744021FF12DE
:103E7B003443755900755A00E55975F003D14F78E5
:103E8B00847F28855A50C242120DC97428255AF5D1
:103E9B005A0559E559B404E0221204BF755B00754D
:103EAB0070027871743912351B1235061235387E53
:103EBB00047D0078847F288D50C242120DB4798422
:103ECB0078707F28E70912351BDFF912351A123586
:103EDB003874282DFDDEDC78701234F91235387405
:103EEB001321FF1204BF755B007570027871744863
:103EFB0012351B1235061234F9123538742131FF85
:103F0B007880515FF51A515FF51B515F515FF51CBE
:103F1B0008515FF519515FF518221204BF755B004C
:103F2B007570027871744712351B123506E51A123B
:103F3B00352FE51B12352F742012352FE51C12354A
:103F4B002F12351AE51912352FE51812352F1235A8
:103F5B001A1234F9123538741321FFC0E01204BF62
:103F6B00755B007570027871744D12351B12350636
:103F7B00D0E012352212351A1234F9123538743E4C
:103F8B0021FFC0E01204BF755B007570027871747D
:103F9B004612351B123506D0E012352212351A1295
:103FAB003538E4120ED98570188571197870E519BA
:103FBB0012352F742E12351BE51812352F12351AA8
:103FCB007F1512354212353874D0120ED71217AD39
:103FDB007F0478707980E70912351BDFF9123538C9
:103FEB0074D4120ED71217AD7F0478707980E7095D
:103FFB0012351BDFF912351A1234F91235387413D6
:10400B000239FF1204BF755B007570027871744141
:10401B0012351B123506123538123AC21235387466
:10402B0000120ED712332A74081233B274081239E5
:10403B00A712351A12353812332A7404120EFF7474
:10404B000C1233B2740C1239A712351A123538749C
:10405B000A120EB97918120CD17870E51A12352F95
:10406B00E51B12352F742012352FE51C12352F123C
:10407B00351A1235387410120ED7123AC61234F99B
:10408B0012353874150239FF9042470206D3843932
:10409B00776D76C23F37C2775FC2763E8437733F08
:1040AB00B18237BF8239B10237CF8373763E82DF5D
:1040BB00F3827776C473760808C44F5F0808C2375B
:1040CB0076837379B18276398776390040760040F2
:1040DB0022734022374082065F825B5F0206390201
:1040EB005B3923397940133173408373383E81F345
:1040FB008239760A73383E00000000003976C237E9
:10410B0077836D38738637733F313F76C43E76764F
:10411B0003C43E76760CC44F567639813701700155
:10412B0046017C015C014801580162824F37837361
:10413B00377D834F397D837637768339663984377C
:10414B003776398437764F76857F79397C3085FDA4
:10415B0037733FDF84395C54F88537F34F77B1827F
:10416B0076BF813982373F8473774F73883779E60F
:10417B000076774FFF84373F5FF3863F66B9003990
:10418B00E6863F7DF60039E68673776D6D795E8541
:10419B007950505C50877C506D077D3F3F81730A8F
:1041AB00797776064F000000000803377366833F6C
:1041BB00317383377966856D38797973863979737D
:1041CB007F3E398479403F37847940763784794014
:1041DB00765F8579407637738479403737857940B8
:1041EB004F7737857940767D6E847940773785793F
:1041FB0040763931847940397684794071388479C5
:10420B00405F778579403F4F3985794076393985DD
:10421B0079407673398579404F777389794071503E
:10422B00407C3E6D6E877940715040763985794080
:10423B0071504088794071504037737689715000C6
:09424B003054003E6D79C279394E
:00000001FF
